:100000000C94080218951895189518951895189538
:1000100018951895189518950C94F501189518953C
:100020001895189518951895189518951895189568
:100030001895189518951895189518951895189558
:100040001895189518951895189518950C94E5011C
:1000500018951895EC0597054605FB04B3046F0445
:100060003004F303BB03850352032303F502CB02E1
:10007000A3027D02590237021702F901DD010804CB
:100080000F0100010F0100010F0408030001080423
:100090000F0100010F0100010F0408040F041002FA
:1000A00012020F08140212010001120100011001D6
:1000B0000001100100010F0100010F0100010D02FC
:1000C0000B040D0212020F080802060208020902C0
:1000D0000B0209020B020D020F02120210020F02A4
:1000E0000D020B020902080206040D0100010D01B8
:1000F00000010D040F0410040F020D020B040D0487
:100100000F040D020B0209040B040D040B0209027B
:10011000080810020F0100010F0100010D0100018C
:100120000D0100010B0100010B01000109020F028A
:100130000D0100010D0100010B0100010B01000187
:10014000090100010901000108020B0200020B0273
:100150000D020F0808040F0100010F0100010F0438
:100160000803000108040F0100010F0100010F0442
:1001700008040F04100212020F08140212010001F9
:100180001201000110010001100100010F01000126
:100190000F0100010D020B040D0212020F080802EC
:1001A0000602080209020B0209020B020D020F02ED
:1001B000120210020F020D020B02090208020604CD
:1001C0000D0100010D0100010D040F0410040F02C8
:1001D0000D020B040D040F040D020B0209040B04A5
:1001E0000D040B020902080810020F0100010F01A3
:1001F00000010D0100010D0100010B0100010B01C7
:10020000000109020F020D0100010D0100010B01A7
:1002100000010B01000109010001090100010802B0
:10022000080409020B020806000208080F08080863
:100230000F0700010F061002120610020F08000837
:100240001408120810080F080D060B020D06120202
:100250000F080008080810080F080D080B0609020F
:1002600008060902060800080B08090808060D021E
:100270000B08090608020606090208040304040420
:100280000604080401040604010404040804030429
:100290000804010408040304080404040804060410
:1002A0000804142012061502140612021006140285
:1002B000120610020F06120210060F020D080008A7
:1002C00001060302040606020806090206060802E1
:1002D00009060602080609020808000812081106A5
:1002E0001402121010060F020D0610020F10120851
:1002F00011061402121010060F020D0610020F1044
:100300000B0609020B060D020F1010060F020D0658
:100310000B020F060D020B0609020D060B02090661
:100320000B020D100F060D020B0609020D060B0243
:10033000090608020B0609020D0609020808000852
:100340009C0101E007BB0DE003BF00E40CBF09E026
:100350000EBD02E109BF789480E090E00EC000E09D
:1003600000936000FC01E158FF4F0491009361008D
:10037000009161000023E1F70296823C02E09007C1
:1003800058F7FC01E258FF4F0491002341F3F89421
:1003900001E000936000FC01E158FF4F04910093DD
:1003A000610000E010E01DBD0CBDFC01E258FF4FF4
:1003B000049110E0000F111FF801EE5AFF4F059154
:1003C00014911BBD0ABD7894D3CF1A930A931FB71B
:1003D00000916100002329F0009161000A950093CB
:1003E00061001FBF0991199118951A930A931FB7BD
:1003F00000916000002329F0C09B02C0C09801C09A
:10040000C09A1FBF09911991189500008895FECFD9
:1004100001EA0DBF00E00EBFC2E8D0E00E941A0260
:10042000002311F00E942A020E94A0010E940502EE
:100430000C94050201E0089520E006D0E9F7089544
:10044000259102D0E9F708952D9301501040202FF7
:10045000212B089588E894E0FC0105911491FC019A
:100460003296A591B491FC01349625913491422F96
:10047000432B19F0F901E4DF01C0DEDF069614E03A
:0E0480008E38910748F30895020060000000D6
:00000001FF
:00000001FF
